:020000040800F2
:10000000000200204D040008B9040008C9040008DB
:1000100091060008A1060008B106000800000000D3
:100020000000000000000000000000000D040008B7
:10003000C106000800000000F10300080B020008E0
:100040000B0200080B0200080B0200080B0200085C
:100050000B0200080B020008F10E0008F10E000868
:10006000F10E0008F10E0008F10E00080B02000866
:100070000B0200080B020008FD0D00080B0200082F
:100080000B020008C50D00080B0200080B02000857
:100090000B0200080B0200080B020008F10E00081A
:1000A0000B0200080B0200080B0200080B020008FC
:1000B0000B0200080B0200080B0200080B020008EC
:1000C0000B0200080B0200080B0200080B020008DC
:1000D0000B0200080B020008B90D0008F10D000822
:1000E000F10E00080B0200080B0200080B020008CA
:1000F0000B0200080B0200080B0200080B020008AC
:100100000B0200080B0200080B0200080B0200089B
:100110000B0200080B0200080B0200080B0200088B
:100120000B0200080B0200080B0200080B0200087B
:100130000B0200080B0200080B0200080B0200086B
:100140000B0200080B0200080B0200080B0200085B
:100150000B0200080B0200080B0200080B0200084B
:100160000B0200080B0200080B0200080B0200083B
:100170000B0200080B0200080B0200080B0200082B
:100180000B0200080B02000800F0AABA704700003A
:1001900070B50C46064600F047F9094B094A1D6840
:1001A0002919914202D8084A914204D20C233360A3
:1001B0004FF0FF3500E0196000F03EF9284670BDB1
:1001C00000020020000002205011002019461046B5
:1001D00000F092BA1946104600F096BA1323036055
:1001E0004FF0FF307047132303604FF0FF3070472C
:1001F000132303604FF0FF30704702294FF00003D4
:1002000003608CBF00200120704700F061BA00003D
:10021000114B70B500241C60104B114D18682E68EE
:1002200000F09CF80F4B53F820301B68A3F1080234
:1002300096420FD026B13179092904BF0A213171C4
:10024000092103F8041C33F9021C074B2A601980AA
:10025000012070BD204670BD880200205C03002094
:1002600090020020980200208C020020082930B55E
:10027000037919D9082B32D842791A4B53F82250F6
:1002800000F108042DB12D68856053F822502C60D0
:1002900000E0846043F82240134C4279012303FAC2
:1002A00002F22368134319E0082B18D945790D4B46
:1002B00053F825203AB11468A2420BBF00222468EB
:1002C00043F825201460427953F822303BB9064C9C
:1002D000012303FA02F2236823EA02032360017177
:1002E00030BD00BF980200205C03002008B50A4B17
:1002F0001B681A79082A02D95B7983420AD900F06F
:100300009EF818B1054B01221A6008BDBDE80840EF
:1003100000F066B808BD00BF9002002088020020EF
:1003200008B500F081F8094B094A1B88094D1BB23A
:10033000002442F82340084A286813682146013BFC
:100340001360FFF793FF2C6000F046F88C0200204A
:10035000D802002090020020940200200023C2074F
:1003600002D440080133FAE718467047134423F0DB
:10037000030310B54FF077321C1F43F8042C6207BB
:1003800042BF4FF0883243F8082CA3F108044FF025
:10039000807304E909000F4B44F80C3C002344F837
:1003A000103C032344F8143C2246022344F8183C32
:1003B000012344F81C3C42F8201D0B2342F8043D65
:1003C000013B032BFAD120466FF0020340F8443D75
:1003D00010BD00BF2103000800F02AF801DFFEE78E
:1003E000024A536843F080535360704700ED00E0C9
:1003F000EFF3098020E9F00F40F804ED02490968A5
:10040000086000F003F8000090020020FFF700FFF2
:1004100004480068016801C9B1E8F00F81F3098858
:100420000047000090020020EFF3108072B6704782
:1004300062B6EFF31080704780F310887047EFF3D7
:100440000580C0B2704770477047000008B5FFF7DD
:10045000FAFF6A46114B1249934202D243F8041B39
:10046000FAE7104A104B11498B4204D252F8040F9C
:1004700043F8040BF8E70E4B0E4A0021934202D2D8
:1004800043F8041BFAE7FFF7DFFF00F047F901F03C
:1004900031FABDE8084000F095B900BF0000002027
:1004A000FEE7FEE71C2C0008000200208802002066
:1004B000880200205011002008B50249042000F0F5
:1004C0004BF900BFC42700080D490E4A0E4B684681
:1004D000904203D8984201D9002102E009468D4696
:1004E000012104207246024202D1EFF3088001E0AC
:1004F000EFF309802DE9F00F6B4600F007F800BF1D
:100500000002002000000220600500202DE9F04FCD
:100510009A46494B8FB093469A6B03925A6B04925A
:100520009F6ADA6A05921A6BDB6B0793434B06925C
:100530001A68434B9A420446884602D0414801F06B
:1005400079FAB8F1000F05D03F48002501F072FAA2
:100550002E4626E094E80E00E068D4F81C9008903F
:100560002069099060690A9019F4007F3748A669EC
:100570000D930CBF04F1200504F124050C920B919E
:1005800001F058FA089B00930BA90EC9304801F0FE
:10059000DFF9CDF8009033460A9A09992D4801F009
:1005A000D7F92D4801F046FA39462C4801F0D0F928
:1005B00005992B4801F0CCF906992A4801F0C8F9B1
:1005C0000799294801F0C4F93A0403D5039927484B
:1005D00001F0BEF93B0603D50499254801F0B8F9AE
:1005E000244801F027FA5946234801F0B1F9B8F13F
:1005F000000F1BD1214801F01DFA3146204801F0BF
:10060000A7F969461F4BC91A03D549421E4801F094
:100610009FF920468268C36801698C4641698E460D
:10062000AD46514691E8F00F4168006801BE174998
:10063000052000F091F800BF00ED00E00000002070
:10064000FEE7FEE7D0270008E62700081528000887
:10065000302800086D280008AB280008B4280008DE
:10066000C4280008D4280008E4280008F42800085A
:100670000429000814290008192900082B2900085A
:100680005C2900085801002084290008B1290008CD
:1006900008B50249062000F05FF800BFC429000831
:1006A00008B50249072000F057F800BFD729000815
:1006B00008B50249082000F04FF800BFE9290008FA
:1006C00008B50249092000F047F800BFFD290008DD
:1006D00008B502490A2000F03FF800BF0F2A0008C1
:1006E000034B044A4FF4E131002000F09FBA00BFF1
:1006F00004020020FD0A00080A460146014800F0F5
:1007000008BA00BF0402002010B50A460C46014694
:10071000002000F035FA204610BD000008B5012188
:10072000094800F081FB0121084800F07DFB012110
:10073000074800F079FB0121064800F075FBBDE891
:10074000084000F025B900BF0D0C02400C0C02401F
:100750000E0C02400F0C024008B50B4B1A680C46F9
:1007600072B9012203281A6003D17146074801F0CB
:10077000EFF82146064801F0EBF8064801F0E8F8EA
:10078000FFF752FE00F0F2F8A00300202F2A000825
:10079000332A00084F2A000808B500F06FFC034810
:1007A00001F0D6F800F036FC002008BD5D2A0008F4
:1007B00008B5034C2368012000F06AF9FAE700BF8E
:1007C000A40A00201FB5FFF72FFE0E4B0E481B6832
:1007D000029300240D4B00930F220C234FF48071E1
:1007E000019400F04DF80A4B0A481B6802930A4B2B
:1007F000009307220C234FF4C061019400F040F8ED
:10080000FFF7EAFD18020020A4030020B10700084A
:100810001C020020A40400209907000808B5FFF777
:1008200003FE094B1B681A79082A07D95A79074B26
:1008300053F8221011B1096843F82210FFF7FCFDAC
:10084000BDE80840FFF7CCBD9002002098020020D0
:1008500038B50B79082B03D908490320FFF77CFF33
:100860004C7901F1080203682BB113F8035CAC4228
:1008700001D31846F7E78B60026038BD1D2A0008D7
:100880000F2A2DE9F74F05468B4691469A462AD8FE
:1008900010F003031BBFC3F10403ED180B46CB1A82
:1008A000303B23F003031AF0080F05EB030405D0D7
:1008B0002A46A24203D212600432FAE72D60019365
:1008C000FFF7B2FD2749019B8046012251F82270B3
:1008D00016B25FB10132212AF8D14046FFF7ACFDD4
:1008E0006FF08A003BE06FF0150038E01D490C986E
:1008F00041F822402A46E6800D99FFF737FD0E9B0E
:10090000194AA3624FF0FF33E3611368206001339B
:100910001AF0010F6562C4F82CB084F805902771B5
:10092000A760E76027616761A7612762136004D051
:1009300001212046FFF79AFC0DE00A212046FFF72F
:1009400095FC1AF0040F06D14046FFF775FD4846A6
:10095000FFF7CCFC02E04046FFF76EFD304603B0E7
:10096000BDE8F08FD80200209402002008B5EFF314
:100970000581C1F3080119B11039044800F0E8FFFE
:1009800000BE042000F084F8FBE700BFAA2A00089C
:1009900010B500F00DFD3B4B002199601A6822F064
:1009A000867222F480321A60D9601A6842F480326A
:1009B0001A601A68334C9003FBD54FF08051002029
:1009C00000F0BEFA304A136843F400431360A36892
:1009D00023F0F003A360A368A360A36823F460433B
:1009E000A360A36843F40043A360A36823F4E05327
:1009F000A360A36843F4A053A3600023636063680B
:100A000043F480036360636843F0080363606368D2
:100A100043F4A843636063686360636843F0E06322
:100A20006360236843F0807323602368154A99014B
:100A3000FBD5164B00211960196841F4007119604B
:100A4000196841F480611960196821F00F0119607B
:100A5000196841F005011960936823F0030393605E
:100A6000936843F002039360936813F0080F054BFB
:100A7000FAD01A6822F001021A601A689207FCD4B0
:100A800010BD00BF0038024000700040003C024032
:100A9000174B93F90010042827D8DFE800F003066D
:100AA0000D15150000221A701FE001221A70114A5C
:100AB000136923F0040316E002221A700E4A136829
:100AC00023F0030313600AE003221A700A4B1A682A
:100AD00042F00E021A605A6842F480725A60054A67
:100AE000136943F00403136130BF0846704700BF29
:100AF0002002002000ED00E00070004038B5044600
:100B0000043000F056FA0546204600F0E9FA28467F
:100B100038BDF8B504460E461746051D3A4631461F
:100B2000284600F031FA20B90121204600F0A8FA49
:100B3000F4E7F8BD4209012300F01F0003FA00F0BA
:100B4000014B43F82200704700E100E008B50B6854
:100B50009B0608D5084B496803EBC002C9B253F89D
:100B6000303050689847054B1B681BB1BDE8084002
:100B7000FFF754BE08BD00BFB80A0020880200205D
:100B80002DE9F84306460C461546FFF758FCDFF8FA
:100B9000849078B118237343254459F80330AC424C
:100BA00006D01A681206FCD514F8012B5A60F6E735
:100BB000BDE8F883134F4FEA8608474401213846C1
:100BC00000F05EFA182202FB06960F48F37C0F49EC
:100BD000072BC8BF0146102003F0070312FB0303D5
:100BE000CA18ADB2D4605560CA58094842F0010233
:100BF000CA504044012100F043FA3846BDE8F843AA
:100C000000F06EBAA80A00200064024000600240B2
:100C1000B00A0020BC2A0008034A182303FB002066
:100C20004168407C00F08CB9BC2A000801282DE9FD
:100C3000F84F05460C4600F2A88018214143554F55
:100C400007EB01087E58544941F8302001EBC00100
:100C50004FF000094B60514B43F820905048012160
:100C600040F8259000EB850000F00AFAD8F808B0AB
:100C70004946584600F0D8F8D8F80C90012148466B
:100C800000F0D2F898F810A05846514600F008F944
:100C90005146484600F004F92846FFF7BDFF98F892
:100CA000113021010BB93F4800E03F48B0FBF1F0A3
:100CB00000F058FC804600F0FDFD84B2204600F0B4
:100CC00055FC0146404600F09BFB4FF0834100F08D
:100CD000A1FC00F0EFFD2401A4B200F00F002043BE
:100CE0008023B06073610023336142F20C03F36030
:100CF000182303FB0573DC7C072C06DC4FF4001182
:100D0000022000F01DF9294905E04FF4800102207E
:100D100000F016F9264904F007031820102210FBF2
:100D2000032200FB057001EB020E037D90F9120017
:100D30005B0643F4823343F050038B50331DCEF8EF
:100D400008300023CEF81430FFF7F4FE062C02DC46
:100D500004F10B000FE0072C04D1164B4FF40042B6
:100D60005A600BE00C2C02DC04F1300003E00F2C85
:100D700004DC04F1370040B2FFF7DCFEF36843F017
:100D80002003F3600020BDE8F88F4FF0FF30BDE88E
:100D9000F88F00BFBC2A0008B80A0020A80A00206B
:100DA000B00A002080DE800200BD01050060024024
:100DB0000064024000E100E001490020FFF7C6BEE8
:100DC0000044004008B5074B07484FF40012DA60B2
:100DD00000F086F9054B1B681BB1BDE80840FFF722
:100DE0001DBD08BD00600240B00A0020880200203E
:100DF00001490120FFF7AABE0048004008B5074B93
:100E000007484FF000629A6000F06AF9054B1B68D2
:100E10001BB1BDE80840FFF701BD08BD00600240FE
:100E2000B40A002088020020F8B50E460125C0F360
:100E3000832120F00F0400F00F0705FA01F10220D2
:100E400000F07EF807FA05F00323216883406FEA7B
:100E5000030C01EA0C012160216806F0030E0EFA72
:100E600000FE4EEA01012160E2680CEA0202E26043
:100E7000E168C6F3810282400A43E2606268BD40D5
:100E800022EA050262606268C6F30016BE4016439D
:100E90006660A268ADB21343A36000206583F8BD0D
:100EA00020F00F0300F00F02F0B51E685700032575
:100EB000BD4026EA05051D601D680224072A04FAC4
:100EC00007F444EA050494BF002201221C6003EBEE
:100ED000820300F007001C6A80000F22824024EA8F
:100EE00002021A621A6A814041EA02001862F0BDE9
:100EF000104B2DE9F0415E691A680F4F164000242F
:100F00004FF001081D4608FA04F31E4206D06B613B
:100F100007EBC40357F83420586890470134102C6D
:100F2000F1D1064B1B681BB1BDE8F041FFF776BC61
:100F3000BDE8F081003C0140C80A00208802002082
:100F400004281CD8DFE800F003080D1217000D4B31
:100F50001A6C1143196412E00A4A536C1943516424
:100F60000DE0084A136B1943116308E0054A536BFF
:100F70001943516303E0034A936B19439163BFF331
:100F80004F8F70470038024070B513467BB18568BB
:100F9000C468A5420BD084680668651C85604568F6
:100FA000013D2C40013B345D01F8014BEEE7D01AC6
:100FB00070BDC368426830B584681B1B934208D07B
:100FC000C3680468013A5D1C1340C560E154002009
:100FD00030BD4FF0FF3030BD0B4B07B519880B48C3
:100FE00009B200F0B5FC684600F0DEF9BDF900106A
:100FF000074800F0ADFC019B694601336846019348
:1010000000F0A4F9EFE700BF8C020020EC2A0008F2
:101010000A2B000810B5124886B000F099FC114B5D
:101020001148198809B200F093FC104B0293002379
:1010300001930F4B0093062208234FF4C0610D4823
:10104000FFF71EFC01230446059304A92246084627
:1010500000F04EF90599084800F07AFCF5E700BF6A
:10106000212B00088C020020442B0008622B000872
:10107000D90F0008480B0020672B000870470000BC
:1010800070B505460C46FFF7CFF92B6806462BB91D
:101090004FF0FF332B60FFF7CFF918E0CCB10F4BC7
:1010A0001C6802212046FFF7E1F82B68013305D1C7
:1010B00004F108032B600023A36003E021462846C7
:1010C000FFF7C6FB3046FFF7B7F9FFF789F90120B4
:1010D00070BDFFF7B1F9204670BD00BF900200203F
:1010E00070B50446FFF7A0F9256806461DB16B1CD4
:1010F00005D100232360BDE87040FFF79DB9284665
:101100000A2150F808392360FFF7B0F8236813B9B3
:101110004FF0FF33236015F8034C3046FFF78CF98E
:101120002046BDE87040FFF7E1B80000F8B505467D
:101130000E46FFF779F9364B364A1B881BB2074635
:1011400052F82320D2F820E0BEF1000F1AD05469E3
:101150009369A34216D9631C5361D3691C4046B9F5
:10116000136933B9631C04D13846FFF765F920468B
:10117000F8BD002C0ADB0EEBC40393E8030085E8FE
:10118000030004E04FF0FF34002EE9D0D56016696B
:1011900076B333681361002C0CDB95695169D36910
:1011A000691A8B42A9BF691C4FF0FF351D40916140
:1011B0000EEBC505736893E8030085E8030016F895
:1011C000043C052B09D0002373600A21A6F1080016
:1011D000FFF74CF816F8034C00E00F243846FFF7F1
:1011E0002BF90E2C02D82046FFF780F80120F8BD1D
:1011F000002C09DA10460321FFF738F83846FFF7CC
:101200001BF9FFF7EDF8F1E73846FFF715F9EDE7C1
:101210008C020020D802002010B583694469C2699D
:101220001C1BA24201DA002010BD5C1C134084612B
:10123000F9D4026A03C902EBC30383E80300012067
:1012400010BD00002DE9F8431E46264B53F82150EF
:10125000254B1B880380074691462DB93046FFF782
:10126000EBF84FF0FF3439E02B79032B28D01F4BDC
:1012700001462846D3F80080FFF7CEFF044638B178
:101280003046FFF7D9F898F80430052B25D122E035
:10129000B9F1000F03D13046FFF7CEF81EE098F801
:1012A0000430C8F80C70052B0CBF05210421404602
:1012B000FEF7DCFF414605F11000FFF7C9FA07E031
:1012C00003C8EB6883E803000A212846FEF7CEFF37
:1012D0003046FFF7B1F8FFF783F801242046BDE858
:1012E000F88300BFD80200208C020020900200206A
:1012F0002DE9F041124F3B881BB2934206460C4643
:10130000154603D10F490320FFF726FAFFF78CF8A3
:101310003A880D4B12B2804653F8227005213846A8
:10132000FEF7A4FF96E80300FC60434684E8030050
:10133000012229462046BDE8F041FFF783BF00BFE8
:101340008C0200201D2A0008D802002070B5044637
:101350000D46FFF769F8B4F90020114B53F822400D
:1013600006461CB90F490320FFF7F6F92379052B30
:1013700004D0FFF761F84FF0FF3070BD95E803002F
:10138000E36883E803000A212046FEF76FFF6479D3
:101390003046FFF751F82046FEF7A8FF012070BD48
:1013A000D80200201D2A00080121FFF7BFBE00005F
:1013B000104BD3F8882042F47002C3F888204FF015
:1013C00000629A60102283F822200021DA7701F16E
:1013D000604000F561400131522980F80023F6D1C8
:1013E0001A6942F010021A615A6942F400725A6195
:1013F000704700BF00ED00E080F0004002E000BF59
:1014000081F0004142001FBF5FEA410392EA030FEF
:101410007FEA226C7FEA236C6AD04FEA1262D2EB39
:101420001363C1BFD218414048404140B8BF5B423E
:10143000192B88BF704710F0004F40F4000020F0D7
:101440007F4018BF404211F0004F41F4000121F0ED
:101450007F4118BF494292EA030F3FD0A2F1010237
:1014600041FA03FC10EB0C00C3F1200301FA03F175
:1014700000F0004302D5494260EB4000B0F5000F98
:1014800013D3B0F1807F06D340084FEA310102F157
:101490000102FE2A51D2B1F1004F40EBC25008BF09
:1014A00020F0010040EA03007047490040EB0000D3
:1014B00010F4000FA2F10102EDD1B0FA80FCACF102
:1014C000080CB2EB0C0200FA0CF0AABF00EBC25001
:1014D00052421843BCBFD0401843704792F0000FEF
:1014E00081F4000106BF80F400000132013BB5E742
:1014F0004FEA41037FEA226C18BF7FEA236C21D0B8
:1015000092EA030F04D092F0000F08BF084670471C
:1015100090EA010F1CBF0020704712F07F4F04D1EA
:10152000400028BF40F00040704712F100723CBFFD
:1015300000F50000704700F0004343F0FE4040F427
:10154000000070477FEA226216BF08467FEA2363E5
:101550000146420206BF5FEA412390EA010F40F4D0
:10156000800070474FF0000304E000BF10F000431C
:1015700048BF40425FEA000C08BF704743F0964303
:1015800001464FF000001CE050EA010208BF70471E
:101590004FF000030AE000BF50EA010208BF7047A5
:1015A00011F0004302D5404261EB41015FEA010CBA
:1015B00002BF84460146002043F0B64308BFA3F1B2
:1015C0008053A3F50003BCFA8CF2083AA3EBC25394
:1015D00010DB01FA02FC634400FA02FCC2F12002B3
:1015E000BCF1004F20FA02F243EB020008BF20F0EA
:1015F0000100704702F1200201FA02FCC2F1200250
:1016000050EA4C0021FA02F243EB020008BF20EA44
:10161000DC7070474FF0FF0C1CEAD0521EBF1CEA72
:10162000D15392EA0C0F93EA0C0F6FD01A4480EA60
:10163000010C400218BF5FEA41211ED04FF0006349
:1016400043EA501043EA5111A0FB01310CF0004075
:10165000B1F5000F3EBF490041EAD3715B0040EA9B
:10166000010062F17F02FD2A1DD8B3F1004F40EB6B
:10167000C25008BF20F00100704790F0000F0CF03E
:10168000004C08BF49024CEA502040EA51207F3A02
:10169000C2BFD2F1FF0340EAC250704740F40000DD
:1016A0004FF00003013A5DDC12F1190FDCBF00F0CE
:1016B00000407047C2F10002410021FA02F1C2F17C
:1016C000200200FA02FC5FEA310040F1000053EA18
:1016D0004C0308BF20EADC70704792F0000F00F066
:1016E000004C02BF400010F4000F013AF9D040EA6C
:1016F0000C0093F0000F01F0004C02BF490011F400
:10170000000F013BF9D041EA0C018FE70CEAD153FD
:1017100092EA0C0F18BF93EA0C0F0AD030F0004C7D
:1017200018BF31F0004CD8D180EA010000F0004031
:10173000704790F0000F17BF90F0004F084691F0EF
:10174000000F91F0004F14D092EA0C0F01D1420229
:101750000FD193EA0C0F03D14B0218BF084608D1F2
:1017600080EA010000F0004040F0FE4040F400003C
:10177000704740F0FE4040F4400070474FF0FF0CCF
:101780001CEAD0521EBF1CEAD15392EA0C0F93EA16
:101790000C0F69D0A2EB030280EA010C49024FEA68
:1017A000402037D04FF0805343EA111143EA101321
:1017B0000CF000408B4238BF5B0042F17D024FF4D9
:1017C000000C8B4224BF5B1A40EA0C00B3EB510FB4
:1017D00024BFA3EB510340EA5C00B3EB910F24BF9D
:1017E000A3EB910340EA9C00B3EBD10F24BFA3EB22
:1017F000D10340EADC001B0118BF5FEA1C1CE0D1EA
:10180000FD2A3FF650AF8B4240EBC25008BF20F09C
:10181000010070470CF0004C4CEA50207F32C2BFF0
:10182000D2F1FF0340EAC250704740F400004FF08D
:101830000003013A37E792F0000F00F0004C02BFBE
:10184000400010F4000F013AF9D040EA0C0093F088
:10185000000F01F0004C02BF490011F4000F013BE2
:10186000F9D041EA0C0195E70CEAD15392EA0C0F4A
:1018700008D142027FF47DAF93EA0C0F7FF470AF82
:10188000084676E793EA0C0F04D14B023FF44CAFC5
:1018900008466EE730F0004C18BF31F0004CCAD15A
:1018A00030F000427FF45CAF31F000437FF43CAF96
:1018B0005FE700BF42000ED2B2F1FE4F0BD34FF0F4
:1018C0009E03B3EB126209D44FEA002343F00043B6
:1018D00023FA02F070474FF00000704712F1610FD9
:1018E00001D1420202D14FF0FF3070474FF00000AB
:1018F000704700BF70B50E4B0E4CE41AA4100025C3
:101900001E46A54204D056F8253098470135F8E721
:10191000FEF73AFC084C094BE41AA41000251E46B9
:10192000A54204D056F8253098470135F8E770BD38
:10193000202C0008202C0008202C0008202C000857
:1019400002440346934202D003F8011BFAE77047B2
:101950000FB40A4B13B51C6824B1A36913B9204610
:1019600000F024FA05AB049AA1680193204600F028
:10197000DBFB02B0BDE8104004B0704784020020D9
:1019800070B50E46054618B183690BB900F00EFA22
:10199000AB69AC6813B9284600F008FA224B9C42A8
:1019A00001D16C6808E0214B9C4201D1AC6803E096
:1019B0001F4B9C4208BFEC68A3891B0701D5236914
:1019C0003BB92146284600F091F810B14FF0FF30A6
:1019D00070BD013EA36816F8011F013BA36091B1E1
:1019E000002B04DAA269934206DB0A2904D023689B
:1019F0005A1C22601970EDE72246284600F022F8B2
:101A00000130E7D1E2E7002B08DA22460A21284616
:101A100000F018F80130D9D00A2070BD23680A20E0
:101A20005A1C2260187070BD8C2B0008AC2B00086B
:101A3000CC2B0008024B01461868FFF7A1BF00BF7E
:101A400084020020F8B50F461446054618B1836994
:101A50000BB900F0ABF9224B9C4201D16C6808E055
:101A6000204B9C4201D1AC6803E01F4B9C4208BF55
:101A7000EC68A369A360A3891A0709D523693BB160
:101A800023682069181A63699842FEB20FDB08E0E8
:101A90002146284600F02AF80028F1D04FF0FF3602
:101AA0001BE02146284600F017F90028F6D1A3686C
:101AB000013BA36023685A1C22601F7063690130D8
:101AC000984204D0A389DB0707D50A2E05D1214609
:101AD000284600F001F90028E0D13046F8BD00BFEB
:101AE0008C2B0008AC2B0008CC2B0008324B70B5B7
:101AF0001D6806460C4625B1AB6913B9284600F0AF
:101B000055F92E4B9C4201D16C6808E02C4B9C424D
:101B100001D1AC6803E02B4B9C4208BFEC68B4F9E0
:101B20000C309AB215071DD4D00602D409223260B7
:101B30003AE0510712D5616B41B104F14403994277
:101B400002D0304600F01CFA00236363A38923F01F
:101B50002403A3810023636023692360A38943F0E6
:101B60000803A38123694BB9A38903F42073B3F558
:101B7000007F03D02146304600F0C6F9A28912F05A
:101B8000010305D00023A36063695B42A36103E006
:101B9000920758BF6369A36023695BB9B4F90C303D
:101BA00003F0800080B230B143F04003A3814FF0D6
:101BB000FF3070BD002070BD840200208C2B000817
:101BC000AC2B0008CC2B00088A892DE9F041054692
:101BD00010070C4659D44B68002B02DC0B6C002B11
:101BE00017DDE66AAEB102F48052002392B22F688C
:101BF0002B600AB1606D15E0216A01232846B047C9
:101C0000411C0FD12B686BB11D2B01D0162B03D1BA
:101C10002F600020BDE8F081A38943F04003A38139
:101C2000BDE8F081A3895A0705D56368C01A636BC4
:101C30000BB1236CC01A00230246E66A216A2846CB
:101C4000B047431CA38906D129681D293AD8214AE7
:101C5000CA40D60736D500226260D90422692260C4
:101C600004D5421C01D12B6803B96065616B2F60FC
:101C70000029CED004F14403994202D0284600F056
:101C80007FF900206063BDE8F0810F69002FC0D0AC
:101C900093070E6808BF4B690F6018BF0023C7EB9E
:101CA00006088B6002E00744C0EB0808B8F1000F9B
:101CB000AFDD43463A46216AA66A2846B047002867
:101CC000F1DCA38943F04003A3814FF0FF30BDE86E
:101CD000F08100BF0100402038B50B6905460C4675
:101CE000DBB118B183690BB900F060F80C4B9C4272
:101CF00001D16C6808E00B4B9C4201D1AC6803E059
:101D0000094B9C4208BFEC68B4F90C302BB121465A
:101D10002846BDE83840FFF757BF002038BD00BF58
:101D20008C2B0008AC2B0008CC2B0008014900F0DC
:101D3000A9B800BFD91C0008002310B504460360F1
:101D40004360836081814366C28103614361836133
:101D5000194608225C30FFF7F3FD054B6362054B23
:101D6000A362054BE362054B2462236310BD00BFF1
:101D700099260008BB260008F3260008172700084C
:101D800070B568234D1E5D430E4605F1740100F0E9
:101D900045F9044640B1002180E842000C30A060C3
:101DA00005F16802FFF7CCFD204670BD836910B5D0
:101DB000044633BB8364C3640365124B124A1B6839
:101DC0008262984204BF0123836100F01FF86060C3
:101DD000204600F01BF8A060204600F017F8002213
:101DE000E06004216068FFF7A7FF01220921A068D5
:101DF000FFF7A2FF02221221E068FFF79DFF0123F7
:101E0000A36110BD882B00082D1D0008F8B51C4BE0
:101E10001E68B369074613B93046FFF7C7FF483657
:101E2000B4687368013B04D4B4F90C507DB16834D4
:101E3000F8E733680BB13668F2E704213846FFF75C
:101E40009FFF30600028F6D10C233B60F8BD4FF6B1
:101E5000FF73E3810123A38165662560A56065604A
:101E600025616561A5610822294604F15C00FFF740
:101E700067FD6563A563A564E5642046F8BD00BF02
:101E8000882B00082DE9F8438046894600F1480474
:101E9000002694B1A5686768013F0CD4AB89012B7B
:101EA00007D9B5F90E30013303D029464046C8475B
:101EB00006436835F0E72468EBE73046BDE8F88371
:101EC00070B50E46B1F90E10002990B014461D46AB
:101ED00006DA00232B60B3891A060ED540230EE0E4
:101EE00001AAFEF785F90028F3DB029A02F470429A
:101EF000A2F500535A425A412A604FF480630020F1
:101F0000236010B070BD00008B8973B59E07054635
:101F10000C4610D401AB6A46FFF7D2FF0099064683
:101F2000284600F07BF868B9B4F90C309A0522D441
:101F300043F00203A38104F14703236023610123DB
:101F4000636118E00D4BAB62A389206043F080030E
:101F5000A381009B6361019B20614BB1B4F90E101A
:101F60002846FEF74AF918B1A38943F00103A3817B
:101F7000A0893043A08102B070BD00BF2D1D0008B4
:101F800038B50546002946D051F8043C0C1F002BFB
:101F9000B8BFE41800F014FC1F4A1368114613B9C7
:101FA0006360146032E0A3420ED92268A018834215
:101FB00004BF18685B68636004BF121822600C607D
:101FC00024E0A24203D813465A68002AF9D11868BF
:101FD0001918A1420BD12168014458188242196096
:101FE00014D1106852685A60014419600EE002D999
:101FF0000C232B600AE021686018824204BF10683D
:102000005268626004BF091821605C602846BDE820
:10201000384000F0D6BB38BD4C11002070B5CD1C47
:1020200025F0030508350C2D38BF0C25002D06467C
:1020300001DBA94202D90C23336046E000F0C0FB6B
:10204000234B1C681A462146A1B10B685B1B0ED4BA
:102050000B2B03D90B60CC18CD501EE08C420DBF6A
:1020600063684B686360136018BF0C4615E00C464C
:102070004968E9E7174C23681BB93046FEF788F832
:10208000206029463046FEF783F8431C18D0C41C54
:1020900024F00304A0420DD12560304600F091FBEE
:1020A00004F10B00231D20F00700C31A0ED05A4282
:1020B000E25070BD211A3046FEF76AF80130EBD1CC
:1020C0000C233360304600F07CFB002070BD00BF65
:1020D0004C110020481100209368013B002B10B4E4
:1020E000936008DA9469A34202DBCBB20A2B02D1D7
:1020F00010BCFFF7A7BC1368581C10601970C8B259
:1021000010BC7047F8B506460F461446D518AC42C9
:1021100008D03A4614F8011B3046FFF7DDFF431C98
:10212000F5D100E00020F8BD2DE9F04F9DB00C4640
:1021300017460393064618B183690BB9FFF736FEBD
:102140007F4B9C4201D1746808E07E4B9C4201D1D8
:10215000B46803E07C4B9C4208BFF468A38918076D
:102160000CD5236953B10023099320238DF829301E
:1021700030238DF82A30DFF8D4B144E021463046D0
:10218000FFF7B4FC0028EED04FF0FF30D5E0039A03
:10219000111D12680391002A80F28C80524243F094
:1021A00002000792049098F800302E2B00F08480F3
:1021B000032298F80010654800F0B2FA48B14023B5
:1021C000CBEB000003FA00F0049B1843049008F1E5
:1021D000010898F800105E488DF82810062208F1D2
:1021E000010700F09DFA002800F09580594B002B64
:1021F00040F08880039B073323F0070308330393E1
:10220000099B53440993B846454615F8013B1BB951
:10221000B8EB07090FD003E0252BF9D0A846F3E768
:102220004B463A4621463046FFF76CFF01307FD0DF
:10223000099B4B44099398F80030002B78D0002379
:102240004FF0FF3204930793059206938DF85330B5
:102250001A930127052229783F4800F061FA05F119
:102260000108049B38B13C4A801A07FA00F0184371
:1022700004904546EEE7D90644BF20228DF853204E
:102280001A0744BF2B228DF853202A782A2A3FF4BC
:102290007EAF079A00210A20A846013598F8003041
:1022A000303B092B03D800FB02320121F4E700295F
:1022B0003FF479AF079276E798F801302A2B0BD1DB
:1022C000039B1A1D1B680392002BB8BF4FF0FF330E
:1022D00008F1020805936BE70023059308F101005C
:1022E00019460A258046013098F80020303A092A1C
:1022F00003D805FB01210123F4E7002B3FF458AF7D
:10230000059155E703AB00932246144B04A93046D0
:10231000AFF3008007E003AB009322460F4B04A904
:10232000304600F093F8B0F1FF3F82467FF468AF8B
:10233000A3895B063FF528AF09981DB0BDE8F08F73
:102340008C2B0008AC2B0008CC2B0008F22B0008CB
:10235000F62B000800000000EC2B00080521000807
:102360002DE9F04791461F460A698B68DDF8208009
:102370009342B8BF1346C9F8003091F8432006468F
:102380000C4612B10133C9F800302368990642BFE8
:10239000D9F800300233C9F80030256815F0060579
:1023A00010D104F1190A07E001235246394630469C
:1023B000C04701301AD00135E368D9F800209B1AD4
:1023C0009D42F1DB94F843302268003318BF0123AB
:1023D00092060FD5E1185A1C302081F843002244A0
:1023E00094F8451082F84310023303E04FF0FF30B9
:1023F000BDE8F08704F1430239463046C04701305A
:10240000F4D02268D9F80050E36802F00602042AEA
:1024100008BF5D1B2269A3680CBF25EAE57500258E
:102420009342C4BF9B1AED184FF000091A344D4572
:1024300009D00123224639463046C0470130D5D065
:1024400009F10109F3E70020BDE8F0872DE9F04329
:1024500017460A7E85B06E2A984606460C460C9BA7
:1024600001F1430E00F0AE8011D8632A22D009D8C2
:10247000002A00F0BB80582A40F0CA8081F845202D
:10248000834955E0642A1ED0692A1CD0C0E0732A13
:1024900000F0B08009D86F2A2ED0702A40F0B880A2
:1024A0000A6842F020020A603EE0752A24D0782AA9
:1024B0003AD0ADE01A6801F14205111D19601368A8
:1024C00084F84230A8E021681A6811F0800F02D029
:1024D000111D196008E011F0400F02F104011960AC
:1024E00002D0B2F9003000E01368002B3CDA2D2254
:1024F0005B4284F8432037E021681A6811F0800FAE
:1025000002D0111D196007E011F0400F02F1040123
:10251000196001D0138800E01368227E5C496F2A9D
:1025200014BF0A2208221BE078225A4984F8452069
:102530002268186812F0800F00F104051D6003D1B5
:10254000550601D5038800E00368D00744BF42F078
:10255000200222601BB9226822F020022260102291
:10256000002084F8430001E049490A226568A5601B
:10257000002D08DB206820F0040020602BB9002D1E
:102580007DD175460CE0002B79D07546B3FBF2F097
:1025900002FB1033CB5C05F8013D03460028F5D162
:1025A000082A0BD12368DA0708D5236962689A42A2
:1025B000DEBF302305F8013C05F1FF35C5EB0E0306
:1025C00023612EE008681A68496910F0800F03D073
:1025D000101D1860136808E010F0400F02F10400AD
:1025E0001860136801D0198000E01960002323618E
:1025F000754616E01A68111D196015686268002199
:10260000284600F08DF808B1401B6060636804E064
:1026100004F1420584F8422001232361002384F859
:102620004330CDF800803B4603AA21463046FFF7F1
:1026300097FE013002D14FF0FF3026E023692A4691
:1026400039463046C0470130F5D023689B0710D586
:10265000002504F1190907E001234A4639463046AE
:10266000C0470130E7D00135E368039A9B1A9D42C9
:10267000F2DBE068039B9842B8BF184605E00B7890
:1026800084F8423004F142058AE705B0BDE8F083E2
:10269000FD2B00080E2C000810B50C46B1F90E10E9
:1026A000FDF794FD0028ABBF636DA3891B1823F4CD
:1026B0008053ACBF6365A38110BD2DE9F0411F4677
:1026C0008B89DB0505460C46164605D502230022FC
:1026D000B1F90E10FDF787FDA389B4F90E1023F4AC
:1026E0008053A38132463B462846BDE8F041FDF7C2
:1026F00071BD10B50C46B1F90E10FDF774FD431C09
:10270000A38915BF606523F4805343F48053A381EC
:1027100018BFA38110BDB1F90E10FDF75FBD000019
:1027200001F0FF01102A2BDB10F0070F08D010F882
:10273000013B013A8B422DD010F0070F42B3F6D186
:10274000F0B441EA012141EA014122F007047FF09F
:1027500000070023F0E80256083C85EA010586EAF6
:10276000010685FA47F5A3FA87F586FA47F6A5FA32
:1027700087F68EB9EED1F0BC01F0FF0102F007023E
:1027800032B110F8013B013A83EA010313B1F8D1E9
:102790000020704701387047002D06BF35460338CA
:1027A000073815F0010F07D1013015F4807F02BF03
:1027B000013015F4C03F0130F0BC0138704700BF54
:1027C000704770474E4D492048414E444C45520099
:1027D0000A49535220737461636B206F7665726689
:1027E0006C6F77656400537461636B20706F696E02
:1027F00074657220636F727275707465642C2072D8
:102800006573657420746F20746F70206F66207319
:102810007461636B000A436F6E746578742062653F
:10282000666F726520686172646661756C743A00E7
:1028300020202072303A2030782530386C780A20F9
:10284000202072313A2030782530386C780A2020E8
:102850002072323A2030782530386C780A202020D7
:1028600072333A2030782530386C780A0020207294
:1028700031323A2030782530386C780A2020206CAC
:10288000723A2030782530386C780A202020706326
:102890003A2030782530386C780A20207073723AEC
:1028A0002030782530386C780A0A004653522F467B
:1028B00041523A0020434653523A2030782530386E
:1028C0006C780A0020484653523A20307825303838
:1028D0006C780A0020444653523A2030782530382C
:1028E0006C780A0020414653523A2030782530381F
:1028F0006C780A0020424641523A20307825303820
:102900006C780A004D4D4641523A203078253038D7
:102910006C780A004D697363004558435F52455413
:102920003A2030782530386C780A00417474656D2F
:102930007074696E6720746F207265636F6E737454
:102940007275637420737461746520666F7220649D
:102950006562756767696E672E2E2E00496E204787
:1029600044423A0A2020736574202470633D307815
:10297000256C780A20206672616D6520300A20205F
:1029800062740A000A49535220737461636B206FAA
:10299000766572666C6F7765642062792061742059
:1029A0006C656173742025642062797465732E0AE6
:1029B0000048415244204641554C542048414E4421
:1029C0004C4552004D454D204D414E414745204814
:1029D000414E444C455200425553204641554C54BB
:1029E0002048414E444C45520055534147452046EE
:1029F00041554C542048414E444C455200444542B8
:102A00005547204D4F4E2048414E444C45520044BE
:102A1000554D4D592048414E444C45520046414980
:102A20004C454420415353455254494F4E2E0025A6
:102A3000700A002A2A2A2052494F54206B65726E70
:102A4000656C2070616E69633A0A25730A0A002A70
:102A50002A2A2068616C7465642E0A0A006D616917
:102A60006E28293A20546869732069732052494FAF
:102A70005421202856657273696F6E3A20323031C6
:102A8000372E30312D646576656C2D3234332D67E9
:102A900039623331322D56616E64726973290A00CE
:102AA00069646C65006D61696E00496E7369646587
:102AB000206973722025640A000000000044004071
:102AC0000000020003000240020002400700260648
:102AD000040000000048004000000400090C02400F
:102AE000080C02400700270304000000326E642037
:102AF00074687265616420737461727465642C20FB
:102B00007069643A202568690A00326E643A204789
:102B10006F74206D73672066726F6D202568690A77
:102B2000005374617274696E672049504320506984
:102B30006E672D706F6E67206578616D706C652EA5
:102B40002E2E0A00317374207468726561642073DC
:102B50007461727465642C207069643A2025686918
:102B60000A00706F6E67003173743A20476F7420EB
:102B70006D7367207769746820636F6E74656E7417
:102B80002025750A0000000024020020000000003B
:102B90000000000000000000000000000000000035
:102BA0000000000000000000000000000000000025
:102BB0000000000000000000000000000000000015
:102BC0000000000000000000000000000000000005
:102BD00000000000000000000000000000000000F5
:102BE000000000000000000000000000232D302B3A
:102BF0002000686C4C0065666745464700303132FE
:102C00003334353637383941424344454600303154
:102C100032333435363738396162636465660000B3
:102C2000541100200000000060030020400000005C
:102C30000000000000000000A02A0008A52A0008EB
:102C4000FF000000000000008C2B0008AC2B0008E7
:102C5000CC2B000800000000000000000000000075
:102C60000000000000000000000000000000000064
:102C70000000000000000000000000000000000054
:102C80000000000000000000000000000000000044
:102C90000000000000000000000000000000000034
:082CA0000000000024020020E6
:040000050800044D9E
:00000001FF
